:020000008F2847
:080008008E2882070834003441
:1000100098349634803486348634073400340F3470
:100020004234403487348734063400340134863413
:10003000A034C034C03405340034003427341034C4
:10004000C234C1340434003400340334E834C334DB
:10005000C33403340034003400346434C434C4344E
:1000600002340034003400340A34C634C534013458
:100070000034003400340134C734C734FF348207FD
:100080000134563446344F342B3449344634023428
:10009000493446342D34563446344F3403345634C0
:1000A00046344F342D3449344634FF348207043407
:1000B00020343234303448347A3405342034323405
:1000C000353448347A3406342034333430344834C8
:1000D0007A34073420343334353448347A340834AD
:1000E00020343434303448347A340A3420343534CB
:1000F000303448347A340C34203436343034483494
:100100007A34103420343834303448347A34143467
:1001100031343034303448347A34FF3409008501C6
:100120008601D501D601D701D801DC0107309F0037
:1001300006170130DA009630DB008316FF3092009C
:10014000FF308500003086002730810083120230A6
:10015000DE000030DF009E220430920017080C38C9
:100160009700DA2422253D248101CD010B1183164D
:1001700085158312292585118316851183125F2128
:100180007321DB0BC828DB0A5C0BC728C8280421B5
:10019000051CCB28B4282225051CCB280730D1000C
:1001A0008724CD219124051CDD28851CD828D3283F
:1001B0002225851CD828DF21D1282225051CDD28F1
:1001C000D10BD1288C24DB21051CF128851CE928C2
:1001D000E4282225851CE928C50BF0280330C5003A
:1001E000E3282225051CF128E023051CFF28851C97
:1001F000FA28F5282225851CFA28E423F12822254F
:10020000051CFF28EC24B428D901A3014D08A40043
:100210004E08A5004F08A6002330C8005530C7007F
:1002200067222B0B2A290130D9005508A300560854
:10023000A4005708A5005808A6002330C800A7014D
:100240004D08A8004E08A9004F08AA002730C70093
:1002500067223329030123042404250426040319F7
:100260005D290230D9000230AA00A701A801A90126
:100270002730C8002330C70067222B0B40294229B2
:10028000D9015D294608AA00A701A801A9012730C4
:10029000C8002330C70067222B0B5D295A0B512958
:1002A00055290130DA0006170023D5014D08D60084
:1002B0004E08D7004F08D8005E29C3220800010865
:1002C000CE000B1D6529CD0A0B11D001D003851579
:1002D000851101084E0203196E297029D00A672979
:1002E0005009CF0008004508C50B8829C500A301A7
:1002F0004D08A4004E08A5004F08A6000310A40C4A
:10030000A50CA60C2330C8004130C7004522C029E7
:10031000C50BA929C500A7014D08A8004E08A900D2
:100320004F08AA000310A80CA90CAA0C4130C70062
:100330002330C8000430A20091222330C8002730A7
:10034000C70067222B0BC029A301A401A501A601A8
:10035000C029C500A3014D08A4004E08A5004F0800
:10036000A6000310A40CA50CA60C2330C800413035
:10037000C70067222B0BC029A301A401A501A60178
:100380002330C7003D30C8000430A2009122422330
:10039000D4015E23B1236E2408004130C7003D30F4
:1003A000C8000430A200912242230130D4005E2311
:1003B000BE236E2408001D22CB236E24080041308A
:1003C000C7003D30C8000430A200912242235108EA
:1003D000083C353E8400800A0A300002031980017F
:1003E00092234130C8003D30C7000430A200912262
:1003F00008000301CA000520CC00FF304C0203199D
:100400001C2A4C0849020319082A4A08073EFA29FF
:100410004A08013E0520A7004A08023E0520A80020
:100420004A08033E0520A9004A08043E0520AA0008
:100430004A08053E0520AB0008000301CA003F2022
:10044000CC00FF304C020319442A4C084502031922
:100450002C2A4A08073E1E2A4A08013E3F20B700C0
:100460004A08023E3F20B8004A08033E3F20B90038
:100470004A08043E3F20BA004A08053E3F20BB0020
:100480004A08063E3F20BC000800AB010430A20031
:100490000330C7070330C807480884002B088007CB
:1004A000AB01031C552A0130AB004708840000084B
:1004B000CA00480884004A088007031C612A0130EA
:1004C000AB00A20B642A0800C703C8034C2AAB0187
:1004D0000430A2000330C7070330C807480884006F
:1004E0002B088002AB010318772A0130AB004708C4
:1004F00084000008CA00480884004A0880020318E3
:10050000832A0130AB00A20B862A0800C703C80368
:100510006E2AAC016722AC0A2B0B8A2A4522AC0357
:100520000800470884000008CA00480884004A08F8
:100530008000C70AC80AA20B912A08005E08CA00F8
:100540005F08CB000630A2000310CB0DCA0DA20B32
:10055000A52A4A0895009712CB0D03189716171273
:10056000CB0D031817160800DE01DF011508DF00A8
:10057000DF0DDE0DDF0DDE0DDF10971ADF145F10CB
:10058000171A5F140800DD01A6080319D62A2330C4
:10059000C800A701A801A9010330AA002730C7009D
:1005A0008922AC080319AC0A2C08DD00B422A7018B
:1005B000A8015E08A9005F08AA002730C800A301AF
:1005C000A401A5015D08A6002330C700D908031DBA
:1005D000EA2AF42A590BF02A45222919FC2AF42A7E
:1005E00067222B0BF42AFC2A0613DA012A08DF0003
:1005F0002908DE009E22FF2A0130DC0006170800D1
:10060000B4225F08A6005E08A500A401A301233060
:10061000C8000030AA000230A900A801A7012730B5
:10062000C70067222B0B252B5F08A6005E08A500DC
:10063000A401A3012330C8000330AA00A901A80126
:10064000A7012730C70045223C2B030123042404C3
:1006500025042604031908005F08A6005E08A5000B
:10066000A401A3012330C8000330AA00A901A801F6
:10067000A7012730C70067222508DE002608DF0013
:100680009E2208003D08A3003E08A4003F08A500E4
:100690004008A6000830C900353084002330C80067
:1006A0002730C7000408CB00F92189224B088400B9
:1006B0002C088000840AC90B522B08003530C70073
:1006C0003330C8000330A20091223830C7003730E1
:1006D000C8000330A20091226E2308000A30A20055
:1006E000333084000730220203197A2B03302202B0
:1006F000031D7F2B2030D408031D2E308C2B0008C7
:100700000319832B8A2BD408031D882B203E8C2BA6
:10071000303E8C2BD40A303E8000A20B902B080078
:10072000840A722BBD01BE01BF01C0010830C9009F
:10073000353084003D30C8002730C7000408CB00A6
:10074000F9214B0884000008D200D2080319AB2B12
:100750004522D203A52B4B088400840AC90B9E2B8B
:1007600008004630AD007230AE006530AF00713029
:10077000B0002E30B1003A30B20008004930AD0070
:100780004630AE007330AF006530B0007430B10059
:100790003A30B20008004D30AD006F30AE0064302A
:1007A000AF006530B0002030B1007330B20065306A
:1007B000B3007430B4003A30B5002030B600080001
:1007C000022428246E2408000301CA005620CC000D
:1007D000FF304C020319FE2B4C0846020319F32B81
:1007E0004A08063EE52B4A08063E5620CC00FF305C
:1007F0004C020319FE2B4C08C600012C03015620A5
:10080000C60008000301CA005620CC00FF304C028D
:100810000319272C4C0846020319112C4A08063EDE
:10082000032C4A08013E5620B7004A08023E5620D3
:10083000B8004A08033E5620B9004A08043E562034
:10084000BA004A08053E5620BB002030BC00080014
:100850004C30AD006F30AE006330AF006B30B00095
:100860002030B1007330B2006530B3007430B40092
:100870003A30B5002030B600080006118610061484
:1008800086178612061606122225061186100614F1
:1008900086178612061606122225061186100614E1
:1008A00086178612061606122225061186100614D1
:1008B000861386120616061222252830A0009824D8
:1008C00022250630A000982422250C30A000982470
:1008D00022250130A0009824222508008030A000A5
:1008E00098240830A2002D3084000008A000B9240C
:1008F000840AA20B752CC030A00098240830A200F6
:100900000008A000B924840AA20B802C08000D3036
:10091000A0009824222508000C30A000982422254D
:1009200008005108C900F9212B08A00098240800EC
:1009300086120611A01B06158610201B86140610B1
:10094000A01A06148613201A8617061606123425D6
:1009500086120611A0190615861020198614061095
:10096000A0180614861320188617061606123425BA
:10097000080086160611A01B06158610201B86147B
:100980000610A01A06148613201A861706160612D9
:10099000342586160611A01906158610201986140E
:1009A0000610A018061486132018861706160612BD
:1009B000342508000630A2004130840083169B01D4
:1009C00083161C141A088312800083169B0A840A5B
:1009D0008312A20BE02C08000630A20041308400F4
:1009E00083169B011C158312000883169A0055304C
:1009F0009D00AA309D009C1483128C1FFD2C8C132B
:100A000083169B0A840A8312A20BF42C0800C530BB
:100A1000D0000A2DD00B092D0B1D112DCD0A0B1165
:100A2000132D0000132D0000152D080007250725A4
:100A30000725072507250725072507250725072556
:100A4000212D08000A30D3001625D30B242D282D84
:100A500008001430D3001625D30B2B2D0330D30000
:100A6000D30B302D000008001430D300000000002C
:060A7000D30B362D080037
:02400E00293F48
:0C420000000000000000000001000500AC
:00000001FF
